:1000000000308A0011290000FF00030E8301A100C7
:100010000A08A0008A010408A2007708A300780853
:10002000A4007908A5007A08A6007B08A70083131E
:1000300083128C308400801E1F288C1A32282208DC
:1000400084002308F7002408F8002508F900260892
:10005000FA002708FB0020088A00210E8300FF0E0B
:100060007F0E09008A110A12BB280A108A100A1191
:1000700082070134F634F634F63401340134F634B0
:10008000F634F634013481347E347E347E34BD342B
:1000900000347E347E347E348134003476347634D9
:1000A0007E347E340034F634F634FE34FE3481344B
:1000B0007E347634763485340034F734F734F734CC
:1000C00000347E347E3400347E347E34BE347E345C
:1000D0007E347E3480340034F734F734EB341C340F
:1000E00000347F347F347F347F340034FE34F03486
:1000F000FE3400340034EF34DF34BF340034813454
:100100007E347E347E3481340034F634F634F63472
:10011000F93481347E347E347E3401340034F63454
:10012000F634F6340934B9347634763476348D3492
:10013000FE34FE340034FE34FE3480347F347F34A9
:100140007F348034C034BF347F34BF34C034803413
:100150007F3480347F3480341C34EB34F734EB3418
:100160001C34F834F7340734F734F8341E346E3462
:1001700076347A347C3483168601553083128600B7
:10018000C9014908133C031CD028283049078400C2
:1001900083138C1EC9281A0880006400C90AC1286C
:1001A0008C128A110A121F28F701F8014608031061
:1001B0004718F707F70CF80CC718F707F70CF80CF7
:1001C0004719F707F70CF80CC719F707F70CF80CE5
:1001D000471AF707F70CF80CC71AF707F70CF80CD3
:1001E000471BF707F70CF80CC71BF707F70CF80CC1
:1001F00000344130840083130008031910290130B2
:10020000F800BF30F7006400F70B0329F80B012951
:100210004A30F700F70B0A2900006400800BFF2822
:100220000034840183131F308305673083169900DF
:10023000A230980090308312980083161F149F14E8
:100240001F159F1107309C0041308312A800A900A0
:10025000AA00AB00AC00AD00AE00AF00B000B10032
:10026000B200B300B400B500B600B700B800B900E2
:10027000BA00BB00FF30BC0083161F149F141F156B
:100280009F1183121F108316091283129412BC123D
:100290003C088316870083123C163C0883168700AF
:1002A0008312BC113C08831687000130831294002E
:1002B0000030831694000108C739083881000F30D8
:1002C000F700073083128101813084008313000816
:1002D000F0390738800064000008F739F719F03961
:1002E0007704800090010030F800920000308316FF
:1002F000920007309C00050864000230F700F70BFD
:100300007F2982291C0883120D1383169D018C16E8
:10031000C03083128B040030F8001F08C7397804FE
:100320009F00BD013D08013C031CD429C0014008C9
:10033000643C031CD2291F151F199C291E08093C67
:1003400003189B29BE013E08093C031CD029BF01AC
:100350003F08043C031CCB293D08C6000A30C700F7
:10036000D4203E087807283E8400831340300002E2
:10037000C500C6000530C700D4203F0878073520E7
:10038000C800831686018312480886000130C10028
:10039000F920BF0AA8290230C100F920BE0AA3290A
:0C03A000C00A9729BD0A92299129630028
:02400E00393F38
:00000001FF
